:020000040000FA
:020000003228A4
:08000800AB0003088301A10015
:100010000A08A20083018A010C1C2A282E0BAE00BC
:10002000003E03190511031D0515B40AAF16341857
:10003000AD0AA50A03192F14B4080319B00AB01A9F
:100040002F16B01F2528B80AB001F0308F00DF301E
:100050008E000C10220883018A0021088300AB0E59
:100060002B0E090083128501073099008316FF23A8
:1000700090001A309F001A3085000C1496018312EC
:100080008512013090000B178B17830121308400FB
:100090004030A000E52085162F12B020D02083200C
:1000A00052204D28AF1D59288512AF10301CAE16B6
:1000B00008002F1D6B288512AF102E0B6B28301DEA
:1000C0006B28B408031D6B282E153808F039031966
:1000D0006B282030AE00AF1E0800AF12AF1C722894
:1000E000B01C762805102F1D851608002608E63C52
:1000F000E630031CA60026092D02031C0800051487
:1001000085122E1508002F1C0800B10A031D962821
:100110002F1E90283608AC00B43CAF150318AF1161
:100120003308A600B301B201B601B5010D309F003E
:10013000AB209F149F189A281E08B2070318B30A11
:1001400005309F00AB209F149F18A4281E08B507F8
:100150000318B60A08000830A000A00BAD2808005C
:10016000A301A801AA01851D231423082406A406BF
:10017000FF39031DA501251DC12824082706A80055
:10018000A706270829052906AA00A806A906270602
:10019000031DA51FCF2827082906AA04A9060800C1
:1001A000AF1908002708013A2805A0000319DC2828
:1001B0000230AF06AE15080029082A050319080009
:1001C0002F15B801B001AE150800A00BE8280800F3
:0601D0008001840AE5280D
:084000000000000000000200B6
:02400E00443E2E
:00000001FF
